:060000000A128A11FC2F18
:100E18008316031306108610061186110612861211
:100E280006138613871307138712071283120313F7
:100E380087170717871607160610861006118611DA
:100E48000612861206138613871F2B2F2C2F412F6D
:100E5800071B2F2F302F412F871A332F342F412F65
:100E6800071A372F382F412F8610061186110612C0
:100E78008612061386130614282F871B442F452F26
:100E88005A2F071F482F492F5A2F871A4C2F4D2F9B
:100E98005A2F071A502F512F5A2F06108614061151
:100EA80086110612861206138613282F871F5D2FB8
:100EB8005E2F732F071F612F622F732F871A652FDD
:100EC800662F732F071A692F6A2F732F0610861043
:100ED800061586110612861206138613282F871BFD
:100EE800762F772F8C2F071B7A2F7B2F8C2F871E1F
:100EF8007E2F7F2F8C2F071A822F832F8C2F06107F
:100F08008610061186150612861206138613282FD8
:100F1800871F8F2F902FA52F071B932F942FA52F57
:100F2800871E972F982FA52F071A9B2F9C2FA52F29
:100F380006108610061186110616861206138613E9
:100F4800282F871BA82FA92FBE2F071FAC2FAD2F27
:100F5800BE2F871EB02FB12FBE2F071AB42FB52F63
:100F6800BE2F061086100611861106128616061365
:100F78008613282F871FC12FC22FD72F071FC52FD2
:100F8800C62FD72F871EC92FCA2FD72F071ACD2FA5
:100F9800CE2FD72F0610861006118611061286123C
:100FA80006178613282F871BDA2FDB2FF02F071B36
:100FB800DE2FDF2FF02F871AE22FE32FF02F071EE7
:100FC800E62FE72FF02F061086100611861106125D
:100FD800861206138617282F06108610061186110A
:100FE8000612861206138613282F0A128A11002861
:080FF80083010A128A110C2F7B
:02400E00BA3FB7
:00000001FF
